:020000040800F2
:10000000E00E0020E90D0008AD030008AF03000872
:10001000B3030008B7030008BB030008000000009A
:10002000000000000000000000000000BF03000806
:10003000C103000800000000C3030008C503000856
:10004000030E0008030E0008030E0008030E00084C
:10005000030E0008030E0008030E0008030E00083C
:10006000030E0008030E0008030E0008030E00082C
:10007000030E0008030E0008030E0008030E00081C
:10008000030E0008030E0008030E0008030E00080C
:10009000030E0008030E0008030E0008030E0008FC
:1000A000030E0008030E0008030E0008030E0008EC
:1000B000030E0008030E0008030E0008030E0008DC
:1000C000030E0008030E0008030E0008030E0008CC
:1000D000030E00085F0D0008030E0008030E000861
:1000E000030E0008030E0008030E0008030E0008AC
:1000F000030E0008030E0008030E0008030E00089C
:10010000030E0008030E0008030E0008030E00088B
:10011000030E0008030E0008030E0008030E00087B
:10012000030E0008030E0008030E0008030E00086B
:1001300000F002F800F05AF80AA090E8000C82449F
:100140008344AAF10107DA4501D100F04FF8AFF27C
:10015000090EBAE80F0013F0010F18BFFB1A43F0A5
:100160000103184728210000482100000A444FF0ED
:10017000000C10F8013B13F0070408BF10F8014B06
:100180001D1108BF10F8015B641E05D010F8016B4B
:10019000641E01F8016BF9D113F0080F1EBF10F8AF
:1001A000014BAD1C0C1B09D16D1E58BF01F801CBD2
:1001B000FAD505E014F8016B01F8016B6D1EF9D555
:1001C0009142D6D37047000000230024002500266A
:1001D000103A28BF78C1FBD8520728BF30C148BFAA
:1001E0000B6070471FB51FBD10B510BD01F013FCAB
:1001F0001146FFF7F7FF00F009F801F031FC03B4F6
:10020000FFF7F2FF03BC00F04FFD000008B500F05F
:10021000DBFC00F043FD00F033FC00F0C7FA2024C3
:1002200000221146104600F0BFFB012200211220DF
:1002300000F0BAFB02220021242000F0B5FB0322CB
:100240000021362000F0B0FB04220021482000F0FD
:10025000ABFB052200215A2000F0A6FB062200215C
:100260006C2000F0A1FB8DE000F0A0FA0022114606
:10027000104600F099FB01220021122000F094FBAF
:1002800002220021242000F08FFB032200213620CF
:1002900000F08AFB04220021482000F085FB0522A3
:1002A00000215A2000F080FB062200216C2000F083
:1002B0007BFB102334A20321062000F051FB102306
:1002C00035A20621002000F04BFB102334A20621AA
:1002D0003F2000F045FB102322460621302000F08D
:1002E000A3FA601CC4B27E2C00DD2024102003235E
:1002F000224606210090672000F0EEFA4FF4FA50F3
:1003000000F09FFC4FF4FA5000F09BFC4FF4FA50C1
:1003100000F097FC4FF4FA5000F093FC4FF4FA50C1
:1003200000F08FFC2048082380220021009008461E
:1003300000F06BFB4FF4FA5000F083FC4FF4FA50DE
:1003400000F07FFC4FF4FA5000F07BFC4FF4FA50C1
:1003500000F077FC14480823802200210090084612
:1003600000F053FB4FF4FA5000F06BFC4FF4FA50DE
:1003700000F067FC4FF4FA5000F063FC4FF4FA50C1
:1003800000F05FFC70E70000302E393627204F4C1C
:10039000454420544553540041534349493A0000D1
:1003A000434F44453A00000000000020704700BF62
:1003B000FEE700BFFEE700BFFEE700BFFEE77047B5
:1003C00070477047704700000CB500200190009006
:1003D0006C48006840F480306A49086000BF694892
:1003E000006800F4003000900198401C01900098D3
:1003F00018B90198B0F5A06FF1D16248006800F417
:10040000003010B10120009001E000200090009821
:10041000012843D15C48006840F010005A49086048
:100420000846006820F0030008600846006840F0B5
:1004300002000860534840685249486008464068D6
:1004400048600846406840F480604860084640685C
:1004500020F47C1048600846406840F4E81048608A
:100460000846006840F08070086000BF454800689A
:1004700000F000700028F9D04248406820F00300E6
:10048000404948600846406840F00200486000BFAC
:100490003C48406800F00C000828F9D10CBD10B5AC
:1004A000FFF792FF10BD10B53648006840F001001C
:1004B000344908600846406834490840314948607A
:1004C00008460068324908402E490860084600681E
:1004D00020F4802008600846406820F4FE00486050
:1004E0004FF41F008860FFF7DAFF4FF000602949E2
:1004F000086010BD10B5002100200022214B5B6870
:1005000003F00C0121B1042906D0082928D107E005
:10051000214B224C236027E01F4B204C236023E01B
:10052000184B5B6803F47010164B5B6803F4803261
:10053000022303EB904022B9194B4343174C23602D
:100540000DE0104B5B6803F4003323B1144B4343BD
:10055000124C236003E0104B4343104C236003E034
:100560000D4B0E4C236000BF00BF064B5B68C3F30E
:1005700003130C4CE15C094B1B68CB40074C236018
:1005800010BD000000100240002002400000FFF8F3
:10059000FFFFF6FE08ED00E000127A0000040020E4
:1005A00000093D000404002010B54FF40051FB4841
:1005B00000F0B5FD4FF40041F84800F0B0FD4FF4F5
:1005C0000041F64800F0ADFD4FF40051F34800F053
:1005D000A8FD10BD10B54FF40051F04800F09FFD8C
:1005E0004FF40041ED4800F09CFD4FF40041EB4812
:1005F00000F095FD10BD10B54FF40051E74800F034
:100600008EFD4FF40051E54800F08BFD10BD2DE943
:10061000F04105462C464FF40051E04800F081FDC2
:1006200000261CE0274607F08007802F04D13902FE
:10063000DA4800F074FD04E04FF40041D74800F0C0
:1006400070FD6006040E4FF40051D44800F067FDC1
:100650004FF40051D14800F064FD701CC6B2082E62
:10066000E0DBBDE8F08110B50446FFF79DFF782080
:10067000FFF7CDFFFFF7BFFF0020FFF7C8FFFFF731
:10068000BAFF2046FFF7C3FFFFF7B5FFFFF7A2FF52
:1006900010BD10B50446FFF787FF7820FFF7B7FFBE
:1006A000FFF7A9FF4020FFF7B2FFFFF7A4FF2046A6
:1006B000FFF7ADFFFFF79FFFFFF78CFF10BD70B591
:1006C00004460D461DB1E0B2FFF7E3FF02E0E0B2E1
:1006D000FFF7C9FF70BD70B50646002418E004F1AD
:1006E000B0000021FFF7EBFF00210220FFF7E7FF3A
:1006F00000211020FFF7E3FF002505E0012130462F
:10070000FFF7DDFF681CC5B2802DF7DB601CC4B2AB
:10071000082CE4DB70BD06E041F6650100E0491EEF
:100720000029FCD1401E0028F6D17047014605E0A3
:10073000002001E0421CD0B27B28FBDB0A00A1F1C3
:100740000101F5D1704770B504460D4605F1B000C2
:100750000021FFF7B4FFA11CC1F3031141F0100009
:100760000021FFF7ACFFA11C01F00F000021FFF7F3
:10077000A6FF70BD10B500218D20FFF7A0FF00215E
:100780001420FFF79CFF0021AF20FFF798FF10BD5A
:1007900010B500218D20FFF792FF00211020FFF7F8
:1007A0008EFF0021AE20FFF78AFF10BD70B5002438
:1007B00018E004F1B0000021FFF781FF00210220C2
:1007C000FFF77DFF00211020FFF779FF002505E0EE
:1007D00001210020FFF773FF681CC5B2802DF7DBF5
:1007E000601CC4B2082CE4DB70BD70B5002418E0B6
:1007F00004F1B0000021FFF762FF00210220FFF7A3
:100800005EFF00211020FFF75AFF002505E00121BF
:100810000846FFF754FF681CC5B2802DF7DB601C4B
:10082000C4B2082CE4DB70BD2DE9F04707460E4644
:100830009046994600250024A8F12000C5B27F2FDC
:1008400002DD0027B01CC6B2B9F1100F24D1314629
:100850003846FFF778FF002408E004EB0511504A02
:10086000505C0121FFF72BFF601CC4B2082CF4DBA5
:10087000701CC1B23846FFF766FF002409E004EBA4
:1008800005110831464A505C0121FFF718FF601C32
:10089000C4B2082CF3DB12E031463846FFF753FFB1
:1008A00000240AE005EB45013E4A02EB4101085DE8
:1008B0000121FFF704FF601CC4B2062CF2DBBDE887
:1008C000F08710B50246012000E050430B00A1F173
:1008D0000104E1B2F9D110BD2DE9FF5F0746914651
:1008E0001E460E9D4FF0000A002435E0301B401ECE
:1008F000C1B20A20FFF7E5FFB9FBF0F00A21B0FB17
:10090000F1F201FB1208BAF1000F14D1701EA042DF
:1009100011DDB8F1000F0CD1AB4605EBDB714910CE
:1009200001FB0471C8B22B4620220199FFF77CFF1E
:1009300010E04FF0010AAB4605EBDB71491001FBFB
:100940000471C8B208F13001CAB22B460199FFF711
:100950006BFF00BF601CC4B2B442C7DBBDE8FF9FA1
:100960002DE9F04104460F461546984600260FE053
:10097000AA5D434639462046FFF756FF04F10800BA
:10098000C4B2782C02DD0024B81CC7B2701CC6B2F9
:10099000A85D0028ECD1BDE8F0810000000C01400A
:1009A0009C1C0008741A00082DE9F04180460E4690
:1009B0001546002731464046FFF7C5FE00240AE0F1
:1009C0007E4A02EB8511085D0121FFF778FE781C55
:1009D000C7B2601CC4B2102CF2DB701CC1B240461E
:1009E000FFF7B1FE00240CE06900491C734A02EBDA
:1009F0004111085D0121FFF762FE781CC7B2601C3F
:100A0000C4B2102CF0DBBDE8F0812DE9F05F0646A2
:100A10000F4690461C46DDF828A04FF0000BE1176A
:100A200004EB5171C910A4EBC10131B92046E117A3
:100A300004EB5171C1F3C70506E02046E11704EB52
:100A40005171C910491CCDB23D4615E029463046CA
:100A5000FFF779FEB1460BE059460BF1010B1AF88E
:100A600001000121FFF72BFE09F1010000F0FF0951
:100A7000C145F1DB681CC5B2A542E7DBBDE8F09FCC
:100A800008B50121202000F059FD0420ADF8000038
:100A900010208DF8030003208DF8020069464848B5
:100AA00000F090FA0421464800F039FB01210820AB
:100AB00000F044FD4FF43C40ADF8000010208DF8EC
:100AC000030003208DF8020069463E4800F07AFAE0
:100AD0004FF43C413B4800F022FBC82000F0B1F845
:100AE0000021AE20FFF7EBFD00210220FFF7E7FD1C
:100AF00000211020FFF7E3FD00214020FFF7DFFD7C
:100B00000021B020FFF7DBFD00218120FFF7D7FD9A
:100B10000021FF20FFF7D3FD0021A120FFF7CFFD2B
:100B20000021A620FFF7CBFD0021A820FFF7C7FD7D
:100B300000213F20FFF7C3FD0021C820FFF7BFFDC4
:100B40000021D320FFF7BBFD00210846FFF7B7FDCA
:100B50000021D520FFF7B3FD00218020FFF7AFFD76
:100B60000021D820FFF7ABFD00210520FFF7A7FDEE
:100B70000021D920FFF7A3FD0021F120FFF79FFD01
:100B80000021DA20FFF79BFD00211220FFF797FDDF
:100B90000021DB20FFF793FD00213020FFF78FFDC0
:100BA00000218D20FFF78BFD00211420FFF787FD2A
:100BB0000021AF20FFF783FD08BD000014040020D2
:100BC00000140140000C014010B56FF0040000F06B
:100BD0007AF92E4800682E49B0FBF1F02D490870D3
:100BE0000846007800EB4001C1EBC0104FF6FF71E2
:100BF00001EAC0002849088010BD0146254A127844
:100C00004A434FF0E0235A6100229A611A46126962
:100C100042F001021A6100BF4FF0E022106900F0BB
:100C200001021AB100F48032002AF5D04FF0E02220
:100C3000126922F001024FF0E0231A6100229A614A
:100C400070470146144A12884A434FF0E0235A6124
:100C500000229A611A46126942F001021A6100BF2D
:100C60004FF0E022106900F001021AB100F4803266
:100C7000002AF5D04FF0E022126922F001024FF075
:100C8000E0231A6100229A617047000000040020EE
:100C900000127A00940700209607002010B54FF448
:100CA000A06000F0C1F810BD014600BF704700BF52
:100CB000494A128802F04002002AF9D0C2B2464BDB
:100CC0001B1D1A80704710B586B00446012144F2FE
:100CD000050000F033FC4FF40070ADF81400032061
:100CE0008DF8160018208DF8170005A93B4800F074
:100CF00069F94FF48060ADF8140004208DF81700F6
:100D000005A9364800F05EF925208DF80000032083
:100D10008DF801008DF8020001208DF8030068466F
:100D200000F087F801940020ADF80800ADF80A0043
:100D3000ADF80C00ADF810000C20ADF80E0001A9C4
:100D4000254800F0A2FC012240F22551224800F083
:100D500034FD0121204800F024FD06B010BD10B57F
:100D600040F225511C4800F00DFE10B31A4800F067
:100D700089FDC4B21A48008800F40040C8B9184878
:100D8000008800F4804060B10A2C03D00020144990
:100D9000088020E01248008840F400401049088094
:100DA00019E00D2C06D10E48008840F480400C4913
:100DB000088010E00A480088C0F30D0009490C546F
:100DC00007480088401C0649088008460088C72854
:100DD00001DD0020088010BD0038014000080140FE
:100DE0009C070020B40700200948804709480047B5
:100DF000FEE7FEE7FEE7FEE7FEE7FEE7FEE7FEE7CB
:100E0000FEE7FEE704480549054A064B7047000027
:100E1000A704000831010008E0080020E00E0020CF
:100E2000E00A0020E00A002031490143314A116004
:100E3000704770B5002100230F22C47804B32D4CF5
:100E4000246804F4E064C4F5E064210AC1F10403F9
:100E5000CA40447804FA03F184781440214309011C
:100E6000254C0678A155047804F01F050124AC40F8
:100E700005786D11AD0005F1E025C5F8004109E0E8
:100E8000047804F01F050124AC401C4D067876114F
:100E900045F8264070BD1A4A0A400243154B1B1FF5
:100EA0001A60704739B1134A121D12680243114B80
:100EB0001B1D1A6006E00F4A121D126882430D4B7B
:100EC0001B1D1A607047042808D14FF0E021096902
:100ED00041F004014FF0E022116107E04FF0E02102
:100EE000096921F004014FF0E02211617047000010
:100EF0000000FA050CED00E000E400E080E100E015
:100F000080FFFF1F10B50446CC48844208D1012160
:100F1000042000F02DFB0021042000F029FB46E016
:100F2000C748844208D10121082000F021FB00219C
:100F3000082000F01DFB3AE0C248844208D101219C
:100F4000102000F015FB0021102000F011FB2EE016
:100F5000BD48844208D10121202000F009FB002176
:100F6000202000F005FB22E0B848844208D101218E
:100F7000402000F0FDFA0021402000F0F9FA16E0D0
:100F8000B348844208D10121802000F0F1FA002109
:100F9000802000F0EDFA0AE0AE48844207D101213A
:100FA000801500F0E5FA0021A01500F0E1FA10BD6F
:100FB00010B50121084600F0DBFA0021012000F005
:100FC000D7FA10BD2DE9F041024600250026002089
:100FD00000230024002791F803C00CF00F0591F8BE
:100FE00003C00CF0100CBCF1000F03D091F802C04C
:100FF0004CEA050591F800C0BCF1000F31D014682F
:1010000000202BE04FF0010C0CFA00F3B1F800C007
:101010000CEA03069E4220D183004FF00F0C0CFA1D
:1010200003F7BC4305FA03FC4CEA040491F803C03F
:10103000BCF1280F06D14FF0010C0CFA00FCC2F8ED
:1010400014C00AE091F803C0BCF1480F05D14FF07D
:10105000010C0CFA00FCC2F810C0401C0828D1D3C7
:101060001460B1F800C0BCF1FF0F34DD54680020FB
:101070002EE000F1080C4FF0010808FA0CF3B1F86B
:1010800000C00CEA03069E4221D183004FF00F0CF2
:101090000CFA03F7BC4305FA03FC4CEA040491F88C
:1010A00003C0BCF1280F05D100F1080C08FA0CF8B8
:1010B000C2F8148091F803C0BCF1480F07D100F1C9
:1010C000080C4FF0010808FA0CF8C2F81080401C18
:1010D0000828CED35460BDE8F0814FF6FF7101803F
:1010E000022181700421C17070470246002093687C
:1010F0000B400BB1012000E00020704701468868DA
:1011000080B2704702460020D3680B400BB101202B
:1011100000E0002070470146C86880B27047016156
:101120007047416170470AB1016100E04161704759
:10113000C16070474FF480320A43826181618261ED
:1011400082698269704702460020434B18684FF657
:101150008073184040EA021008433F4B1860704704
:101160003E49C8617047F0B50A46002300240021BB
:10117000002500F00046B6F1004F02D1364EF1696D
:1011800001E0354E7168C0F3034583B200F44016A8
:10119000B6F5401F08D121F070612F4E766826F019
:1011A00070662D4F7E6012E000F48016B6F5801F49
:1011B00006D1032606FA05F4A14341F0706106E06A
:1011C000460D360103FA06F6B14341F0706122B1D3
:1011D000460D360103FA06F6314300F00046B6F13B
:1011E000004F02D11C4EF16101E01B4E7160F0BD59
:1011F00030B500228B071C0F0F2303FA04F2164BA5
:1012000008338C1053F824309343134C08348D105A
:1012100044F8253023468C1053F824308C07240FD3
:1012200000FA04F423430C4C08348D1044F82530A4
:1012300030BD0A49DC3108607047000000080140F9
:10124000000C014000100140001401400018014052
:10125000001C01400020014000000140000020422D
:10126000DF48006840F00100DD490860084640683A
:10127000DC490840DA49486008460068DA49084015
:10128000D74908600846006820F4802008600846B6
:10129000406820F4FE0048604FF41F0088607047EB
:1012A000CF49096821F48031CD4A1160114609689F
:1012B00021F480211160B0F5803F03D0B0F5802F7C
:1012C0000ED106E0C649096841F48031C44A116074
:1012D00007E0C349096841F4A021C14A116000E058
:1012E00000BF00BF704710B5014600220023002058
:1012F0004A11012A02D1BA4C236806E0022A02D11F
:10130000B74C236A01E0B64C636A01F01F02012466
:1013100094401C400CB1012000E0002010BD38B505
:10132000002000900024002500BF3120FFF7DBFFE4
:1013300005460098401C00900098B0F5A06F01D0C1
:10134000002DF2D03120FFF7CEFF08B1012400E0DC
:101350000024204638BD01460020A14A106820F034
:10136000F80040EAC10010607047A049086070476B
:10137000024600209A4B586820F47C1042EA010390
:101380001843974B58607047984908667047014664
:101390000020934A506820F00300084350607047D3
:1013A0008F48406800F00C007047014600208C4ACE
:1013B000506820F0F000084350607047014600205C
:1013C000874A506820F4E060084350607047014647
:1013D0000020834A506820F4605040EAC100506009
:1013E000704729B17E4A527A02437D4B5A7204E01B
:1013F0007B4A527A82437A4B5A7270477B49D83182
:101400000860704701460020754A506820F440404B
:101410000843506070470021714A20321170704AB1
:1014200082F82010012802D004280AD104E001210A
:101430006B4A2032117005E00521694A2032117093
:1014400000E000BF00BF7047694908607047644909
:10145000096A0143624A116270476549443908606C
:10146000704730B500210022002400235C4D6D68D8
:1014700005F00C0121B1042905D0082923D105E08C
:101480005C4D056022E05B4D05601FE0544D6D68CA
:1014900005F47012524D6D6805F48034022505EB99
:1014A00092421CB9544D554305600BE04C4D6D689C
:1014B00005F400351DB1504D5543056002E04D4D1A
:1014C0005543056002E04B4D056000BF00BF444D31
:1014D0006D6805F0F0010909484D6B5C0568DD4059
:1014E00045603F4D6D6805F4E061090A434D6B5C52
:1014F0004568DD4085603A4D6D6805F46051C90A64
:101500003E4D6B5C4568DD40C560354D6D6805F44A
:101510004041890B3A4D6B5CC568B5FBF3F505613D
:1015200030BD29B12E4A526902432D4B5A6104E065
:101530002B4A526982432A4B5A61704729B1284A83
:1015400092690243264B9A6104E0254A92698243DC
:10155000234B9A61704729B1214AD2690243204B3B
:10156000DA6104E01E4AD26982431D4BDA6170479A
:1015700029B11B4AD2680243194BDA6004E0184AC9
:10158000D2688243164BDA60704729B1144A126957
:101590000243134B1A6104E0114A12698243104B53
:1015A0001A61704712494039086070470F49C86492
:1015B00070470B49C87170470948406A40F0807015
:1015C00007494862704701460020054A92680A4070
:1015D0000AB1012000E0002070470149887270477D
:1015E000001002400000FFF8FFFFF6FE000042423C
:1015F0008004424200127A0000093D009E0700204C
:10160000AE07002010B50446FB48844209D10121F1
:101610008803FFF7ADFF00214FF48040FFF7A8FFDC
:1016200032E0F648844209D101214804FFF7ADFFBA
:1016300000214FF40030FFF7A8FF25E0F048844276
:1016400009D101218804FFF7A0FF00214FF4802079
:10165000FFF79BFF18E0EB48844209D10121C80441
:10166000FFF793FF00214FF40020FFF78EFF0BE000
:10167000E548844208D101210805FFF786FF0021D3
:101680004FF48010FFF781FF10BD2DE9F04786B0C1
:1016900005460E460024A24600BFA1460027B08999
:1016A00000B100BF2F462C8A4CF6FF700440F08832
:1016B00004432C82AC894EF6F3100440B088318983
:1016C0000843718908430443AC81AC8A4FF6FF405C
:1016D0000440B0890443AC8201A8FFF7C2FEC648AB
:1016E000874202D1DDF810A001E0DDF80CA0A88946
:1016F00000F4004040B10AEBCA0000EB0A10316868
:101700004900B0FBF1F807E00AEBCA0000EB0A1051
:1017100031688900B0FBF1F86420B8FBF0F00401F7
:101720002009642101FB1089A88900F4004040B120
:10173000322000EBC900B0FBF1F000F007000443D9
:1017400008E0322000EB09106421B0FBF1F000F05A
:101750000F0004432C8106B0BDE8F0874FF416510A
:10176000016000218180C18001810C214181002123
:101770008181704710B502460020108A4FF2FF03A6
:1017800018400B884C8823438C882343CC88234300
:101790001843108210BD0021018041808180C180EA
:1017A000704721B1828942F40052828104E082892B
:1017B0004DF6FF731A4082817047F0B5034600244E
:1017C00000260025002040F66A17B94200D100BF6C
:1017D0001846C1F3421401F01F06012707FA06F567
:1017E000012C01D10C3004E0022C01D1103000E0BA
:1017F00014301AB107682F43076002E00768AF434F
:101800000760F0BD1AB1838A0B43838202E0838AAA
:101810008B4383827047028A4FF6F0731A4002822C
:10182000028A0A430282704782894FF2FF731A408C
:10183000828182890A438281704721B1828942F084
:101840000202828104E082894FF6FD731A40828190
:101850007047028A4FF6DF731A400282028A0A43F7
:101860000282704721B1028A42F48042028204E07F
:10187000028A4BF6FF731A4002827047C1F30802D6
:101880008280704701468888C0F3080070478189CC
:1018900041F0010181817047028BD2B20283028B39
:1018A00042EA012202837047028B02F47F420283E4
:1018B000028B0A430283704721B1828A42F02002E0
:1018C000828204E0828A4FF6DF731A408282704778
:1018D00021B1828A42F01002828204E0828A4FF6AD
:1018E000EF731A408282704721B1828A42F0080267
:1018F000828204E0828A4FF6F7731A408282704730
:1019000021B1828942F40042828103E08289C2F3DC
:101910000E028281704721B1828A42F40062828283
:1019200004E0828A4FF2FF731A4082827047828AF3
:101930004FF6FB731A408282828A0A438282704782
:1019400021B1828A42F00202828204E0828A4FF64A
:10195000FD731A408282704702460020B1F5007F75
:1019600000D100BF13880B400BB1012000E0002024
:10197000704701F40072B2F5007F00D100BFCA4386
:101980000280704770B50246002400230025002025
:1019900040F66A16B14200D100BFC1F3421501F012
:1019A0001F03012606FA03F3012D02D19689334065
:1019B00006E0022D02D1168A334001E0968A3340B8
:1019C0000C12012606FA04F41688344013B10CB147
:1019D000012000E0002070BD10B50022002340F679
:1019E0006A14A14200D100BF0A1201249440A3B29C
:1019F000DC43048010BD000000380140004400407A
:101A000000480040004C00400050004070477047C4
:101A1000704770477047754600F028F8AE460500DD
:101A20006946534620F00700854618B020B5FFF7F9
:101A3000E9F9BDE820404FF000064FF000074FF0F5
:101A400000084FF0000B21F00701AC46ACE8C009DC
:101A5000ACE8C009ACE8C009ACE8C0098D467047E5
:101A60000446AFF300802046FEF7C9FB00487047EC
:101A70007C0800200000000000000000002F000093
:101A800000000700070000147F147F1400242A7F41
:101A90002A120062640813230036495522500000C0
:101AA0000503000000001C224100000041221C0030
:101AB0000014083E08140008083E0808000000A0B2
:101AC00060000008080808080000606000000020AE
:101AD00010080402003E5149453E0000427F40008C
:101AE000004261514946002141454B310018141212
:101AF0007F10002745454539003C4A4949300001DF
:101B00007109050300364949493600064949291E2D
:101B1000000036360000000056360000000814228F
:101B2000410000141414141400004122140800028F
:101B30000151090600324959513E007C1211127CB4
:101B4000007F49494936003E41414122007F4141E1
:101B5000221C007F49494941007F09090901003ED3
:101B60004149497A007F0808087F0000417F410011
:101B7000002040413F01007F08142241007F404087
:101B80004040007F020C027F007F0408107F003E6F
:101B90004141413E007F09090906003E4151215E55
:101BA000007F091929460046494949310001017F52
:101BB0000101003F4040403F001F2040201F003FE8
:101BC0004038403F0063140814630007087008079A
:101BD00000615149454300007F41410000552A55AD
:101BE0002A55000041417F00000402010204004028
:101BF000404040400000010204000020545454784A
:101C0000007F484444380038444444200038444469
:101C1000487F00385454541800087E090102001807
:101C2000A4A4A47C007F080404780000447D400044
:101C3000004080847D00007F102844000000417F28
:101C40004000007C04180478007C08040478003804
:101C50004444443800FC242424180018242418FC8C
:101C6000007C0804040800485454542000043F44F5
:101C70004020003C4040207C001C2040201C003CB8
:101C80004030403C004428102844001CA0A0A07C08
:101C9000004464544C441414141414140000000040
:101CA000000000000000000000000000000000F83C
:101CB00000000000000000333000000000100C069F
:101CC000100C0600000000000000000040C078403A
:101CD000C0784000043F04043F040400007088FC06
:101CE00008300000001820FF211E0000F008F0005E
:101CF000E018000000211C031E211E0000F00888CF
:101D0000700000001E2123241927211010160E0038
:101D1000000000000000000000000000000000E0E3
:101D200018040200000000071820400000020418F8
:101D3000E00000000040201807000000404080F054
:101D4000804040000202010F01020200000000F08A
:101D5000000000000101011F01010100000000005E
:101D60000000000080B070000000000000000000D3
:101D7000000000000001010101010101000000005C
:101D800000000000003030000000000000000000F3
:101D900080601804006018060100000000E01008D0
:101DA0000810E000000F102020100F00001010F8A5
:101DB000000000000020203F2020000000700808E4
:101DC0000888700000302824222130000030088864
:101DD000884830000018202020110E000000C0208C
:101DE00010F8000000070424243F240000F80888AD
:101DF000880808000019212020110E0000E010883A
:101E000088180000000F112020110E00003808086B
:101E1000C83808000000003F00000000007088087B
:101E200008887000001C222121221C0000E01008FC
:101E30000810E0000000312222110F00000000C055
:101E4000C0000000000000303000000000000080F2
:101E500000000000000080600000000000008040E2
:101E600020100800000102040810200040404040FB
:101E7000404040000404040404040400000810204E
:101E80004080000000201008040201000070480893
:101E90000808F0000000003036010000C030C828FB
:101EA000E810E0000718272423140B000000C038B6
:101EB000E0000000203C23020227382008F8888830
:101EC00088700000203F202020110E00C03008083C
:101ED00008083800071820202010080008F8080813
:101EE0000810E000203F202020100F0008F888880C
:101EF000E8081000203F20202320180008F88888D8
:101F0000E8081000203F200003000000C03008084F
:101F10000838000007182020221E020008F80800D8
:101F20000008F808203F210101213F20000808F89F
:101F3000080800000020203F2020000000000808C2
:101F4000F8080800C08080807F00000008F888C082
:101F500028180800203F20012638200008F8080033
:101F600000000000203F20202020300008F8F8006A
:101F7000F8F80800203F003F003F200008F830C07C
:101F80000008F808203F200007183F00E01008086C
:101F90000810E0000F10202020100F0008F808089B
:101FA0000808F000203F210101010000E0100808AE
:101FB0000810E0000F18242438504F0008F88888D3
:101FC00088887000203F2000030C302000708808B3
:101FD000080838000038202121221C00180808F8C1
:101FE000080818000000203F2000000008F8080042
:101FF0000008F808001F202020201F000878880013
:1020000000C83808000007380E010000F80800F882
:102010000008F800033C0700073C0300081868802C
:102020008068180820302C03032C30200838C800A2
:10203000C83808000000203F2000000010080808F1
:10204000C83808002038262120201800000000FE93
:10205000020202000000007F40404000000C30C03F
:1020600000000000000000010638C000000202026B
:10207000FE000000004040407F000000000004021D
:102080000202040000000000000000000000000048
:102090000000000080808080808080800002020438
:1020A0000000000000000000000000000000808030
:1020B000808000000019242222223F2008F800809E
:1020C00080000000003F112020110E000000008061
:1020D00080800000000E11202020110000000080F0
:1020E0008088F800000E112020103F200000808022
:1020F00080800000001F222222221300008080F036
:10210000888888180020203F202000000000808060
:1021100080808000006B94949493600008F80080A5
:1021200080800000203F210000203F200080989800
:10213000000000000020203F202000000000008060
:102140009898000000C08080807F000008F80000A0
:1021500080808000203F24022D302000000808F8F5
:10216000000000000020203F2020000080808080B0
:1021700080808000203F20003F20003F8080008042
:1021800080800000203F210000203F200000808050
:1021900080800000001F202020201F008080008001
:1021A0008000000080FFA12020110E0000000080B0
:1021B00080808000000E112020A0FF8080808000A1
:1021C0008080800020203F212000010000008080CE
:1021D000808080000033242424241900008080E0C3
:1021E000808000000000001F202000008080000090
:1021F00000808000001F202020103F208080800071
:102200000080808000010E30080601008080008080
:10221000008080800F300C030C300F0000808000A5
:10222000808080000020312E0E31200080808000D0
:102230000080808080818E70180601000080808080
:10224000808080000021302C22213000000000001E
:10225000807C020200000000003F404000000000BF
:10226000FF00000000000000FF0000000002027CF0
:10227000800000000040403F000000000006010117
:10228000020204040000000000000000AC2200086C
:1022900000000020B40700006C01000814250008AD
:1022A000B40700202C070000C80100081116060A18
:1022B000FE0AC612E012F062F84EFE7DBBC7EF01C7
:1022C000053EC7BB7DFE300D080CFEFE0C082060ED
:1022D000FEFE60208F7848FE82BABA0309135EAA18
:1022E0000101017E6CFEFF0301CBFFFF0F39BBEC48
:1022F000C0C0C0271918F92701392975990B6CFF3F
:10230000FF0C01491A0C22E1E1E12701396C0F1F92
:102310001801FB1F0F0F092E270136168C422212BF
:102320000C26FC020202FC3304FE16205844FE4038
:102330002A10015912491E4912A92A0123300A24E0
:10234000A42E24E4242EA424C00AF84A4C48F848B9
:102350004C4AF82A01013907490D5915991F991856
:10236000091412712BC020A1AB20C00A11300A122F
:102370000A07027F02070A121E0B0A0A0A7F0402DA
:10238000560B980A1F2040404050205F800A117C65
:10239000A24A04B92008020304060708092AF09F8C
:1023A0002AFF050215F01B0F04012AFF0502130F77
:1023B000195C1E5F55555575041A5F0C09112108EB
:1023C0000C11200F094989790909090F201F112FC4
:1023D000FE02424ACA4A0304134202FE000E14FFE0
:1023E00040504C4340404F50505C40FF1BF8880128
:1023F0002AFF050215F81B1F08012A7F200B109FDA
:1024000080E23B808201000916E2A2928A868280E5
:1024100080041840807F172424A4FEA3221B22CC12
:10242000AA011415080601FF2B0104010511FF0282
:1024300002025808101010FF109008C3021108087B
:102440000F100444827F01808040432C1028468175
:10245000A018094040484848C8784F060515484824
:1024600040400009150312122222528A063C1060D5
:1024700080BA19040B11C030FB1E404043407F0658
:102480001C7F424106094FC02941080B1110D03072
:10249000FF30D0121C10101F3D080402019E0D11C8
:1024A00001020408211116FE222222FE0712FE82DA
:1024B0008292A29E100880601F0242827F0F11FF4D
:1024C000402F102C438011000B1490884C57A424EB
:1024D00054548C84180801018042221A07441D427A
:1024E0003E01018AF9E1000D14E4242CB4252624D0
:1024F000B42C24E404180AFF02011E1212121E4119
:102500008601202D010203040420090607080902A0
:0425100004060800B5
:0400000508000131BD
:00000001FF
